:030000000219FDE5
:03000B000200A848
:03002B000201646B
:03005B000202EEB0
:030073000202D4B2
:1000800002030406080C10182030406080040608A3
:100090000C10182030406080A0C000070F1F3F05E3
:1000A000050D050305030302C2AFC0D0C0E0206206
:1000B00017E5256002E473E525F4F58A758B00D217
:1000C00062D0E0D0D0D2AF3285268AC262E526F473
:1000D0006036306803207210758B00D0E0D0D0C23B
:1000E00090C287C291D2AF32C290C287C291206EB5
:1000F0000D20660A7401D5E0FDE57EF45290758B03
:1001000000D0E0D0D0D2AF32758A00C28DD2620169
:10011000FE01B7306805206602D29001B73068054D
:10012000206602D28701B7306805206602D29101AD
:10013000B7D29630680A2066077405D5E0FDD290E4
:1001400001B7D29430680A2066077405D5E0FDD265
:100150008701B7D29530680A2066077405D5E0FD9F
:10016000D29101B7C2AFC2AD53E6EFC0D0C0E0D26A
:10017000D3D2AFC2CEE52A6007207449152A21C523
:100180007800790020742EE580307E01F430E6029C
:1001900078FF53DACF207E0343DA20307E0343DA40
:1001A00010C2D8C271E580307E01F430E60279FFDA
:1001B000C3E89970CB306103752A18207403752A3F
:1001C00018885FD27020740DE52B6004152B21D5A3
:1001D00043DA01C2D82070024137A85F206102C211
:1001E00070207431C3E894F0400374F0F8E8C4540C
:1001F0000F28F87984B703024115C313C31387216D
:10020000200802C313200A06C3C898F8411528F82D
:10021000500374FFF8C3E895685003E568F8882236
:10022000E52D54066011E533C313C31324062522BC
:10023000F52250037522FF852224A824C3E52495C6
:10024000644002A8648825E5697002417BC3E8AA7E
:10025000699A5003E8FAE4F9EAC333FBE56BF45B0F
:1002600029400D256AF8E56A6002156A400B417B5A
:100270000AC3E56A9A5002056A78FF8826C26EC3EF
:10028000E52694F84002D26EC3E52594404002D2A0
:100290006420CF0AD0E0D0D043E610D2AD32C2CF36
:1002A000053A7801E52A6005307402152AC3E55F36
:1002B0009401400575620041CA756300756C00E5E4
:1002C000622401F56250037562FFD0E0D0D043E6AE
:1002D00010D2AD32C2AFC0D053E67FC2607591007C
:1002E000855694855795759104D0D0D2AF32C2AF60
:1002F00053E6EFC2ADC0D0C0E0C0F0D2D3D2AFA8B9
:10030000FBA9FCC2D8307102615553DACF207E03BD
:1003100043DA10307E0343DA20D271E580307E016B
:10032000F420E602612C88278928A17C53DACF20AB
:100330007E0343DA20307E0343DA10C2D8C2713024
:100340007402A1687800E580307E01F430E602A1F5
:1003500068885FA15053DACF207E0343DA20307ED5
:100360000343DA10C271206102812E53DACF207E5E
:100370000343DA10307E0343DA20C2D8D271885AA0
:10038000895BC3E89558F8E99559F97B007E087AAE
:1003900000C3E8948CE994005005755E00812088C4
:1003A0002178A2E6A8216055C3E894C8E9940050DA
:1003B00008E4D2E4FB7A0A61FBC3E89468E994019B
:1003C0005008E4D2E3FB7A0F61FBC3E894D0E994D0
:1003D000025008E4D2E2FB7A1E61FBC3E894A0E974
:1003E00094055008E4D2E1FB7A3C61FBC3E89498A1
:1003F000E994085008E4D2E0FB7A787E00C3E895DF
:100400005CFCE9955DFD30E70AECF42401FCEDF4B9
:100410003400FD755E00C3EC9AED9E5003755E01DD
:10042000885C895D855A58855B597802A150C3E87C
:100430009527F8E99528F9307C02A134307B02A198
:1004400034307A02A12D2075028151E9FDE8FC814A
:1004500070E9C313F9E813F8307902A12DE9C31349
:10046000F9E813F8307802A12DE9C313FDE813FC75
:0F047000206126C3EC941CED940240028187EDBD
:10047F007018C3EC94C850120529C3E529940A508B
:10048F0002A168755F00D270A168E5296002152985
:10049F007888E6F97400207F087896B90302789E71
:1004AF00E624FAFEE43400FFC3EC9EFCED9FFD92C0
:1004BF0008B90310A2085007207609D27681D330ED
:1004CF007602C276A2085016B9030DECF42401FC93
:1004DF00EDF43400FD0204ED78007900A134B90386
:1004EF0015EC33FCED33FDC3EC940AFCED9400FDE9
:1004FF0050047C007D00C3EC94FFED94004006781F
:10050F00FF7900A134EC8575F0A4C5F0A2F733F89C
:10051F007900400302055078FF7900020550E9C3C6
:10052F0013F9E813F8307C0EE9600278FFC3E81383
:10053F0038F8E43400F9C3E894FFE99400400278F6
:10054F00FF885FD270206102A168741FF4552F4B92
:10055F00F52FC274EB7002D274752A1830740375BC
:10056F002A0A306102A17C20740353DAFE2074033F
:10057F00752B06D0F0D0E0D0D0D2AD43E610327953
:10058F00010205AC79030205AC790A0205AC791EAC
:10059F000205AC79640205AC79C80205AC7817E4A2
:1005AF00D5E0FDD8FAD9F6227A147B780205D37AF2
:1005BF00107B8C0205D37A0D7BB40205D37A0B7BAB
:1005CF00C80205D37902B27DE4D294D5E0FDD2877B
:1005DF00D5E0FDC287D5E0FDC294D5E0FDD290E510
:1005EF0076D5E0FDC2907496D5E0FDD9D9EAF8D55D
:1005FF00E0FDD8FBDBCED29422C37C007D0075F0EA
:10060F000005F0EA33FAEB33FB50F6EB13FBEA137A
:10061F00FAC3E9FFE8FEE89AF8E99BF95004EFF90D
:10062F00EEF8B3EC33FCED33FDD5F0DFEDF9ECF87C
:10063F0022E889F08A20D2D4F8A9F07B0030F70B9A
:10064F007BFFF42401F8E9F43400F9E88520F0A4E5
:10065F00ADF0F8E98520F0A4AFF0FEED2EF97400AF
:10066F003FFA7C04C3EA13FAE913F9E813F8DCF450
:10067F008BF030F70AE8F42401F8E9F43400F9E8D4
:10068F0089F0C2D4F8A9F02222C3E54113F9E5405D
:10069F0013F8C3E54598F8E54699F9500CC3E8946B
:1006AF0080E994FF40160206CFC3E8947FE99400D7
:1006BF0050030206CF787F79000206CF788079FF4A
:1006CF00884A894B22E54A2547F8E54B3548F98595
:1006DF004B20E4300701F43549FA30E709C3EA94B7
:1006EF00F0401502070DC3EA940F500302070D786F
:1006FF00FF79FF7A0F02070D780079007AF0C3E5D2
:10070F00249564500AC374019524500B02072BE5FE
:10071F004B20E70E02072BE54B30E7068847894849
:10072F008A492278A4E6FAC3E54A33F8E54B33F950
:10073F00D140E930E70BC3E89480E994FF4013E11F
:10074F0065C3E8947FE994005002E165787F7900F2
:10075F00E165788079FFE820E715C3E52398F84035
:10076F0009C3E89401400302078C780102078CE863
:10077F00F424012523F8400302078C78FF884C22CC
:10078F0078A5E6FAA848A949D140E930E70CC3E8B3
:10079F009401E994FF40160207C0C3E894FFE9945F
:1007AF000050030207C078FF79000207C078017973
:1007BF00FFE920E715C3E54C98F84009C3E8940119
:1007CF0040030207E778010207E7E8F42401254C0C
:1007DF00F840030207E778FF88242278FFC26420DD
:1007EF00693D206A12D264C3E541940A4009C3E50A
:1007FF002594405002C26479A1E76023E541601F50
:10080F0074FF8541F0848539F0306A0375F005A4D3
:10081F00F8C5F0600278FFC3E895675002A86788B3
:10082F006622C3E5409440E5419401E56650031408
:10083F000142046002F5662202084A2275E89022FE
:10084F007883E6FFE5E820ECF7A8BDA9BE0573C3E2
:10085F00E57394084052757300E9FA79A0E7604494
:0E086F00EA7007E574601B020885C3E8957403
:10087D006010E5745006600C140208910460F902D2
:10088D000891E574F574C39467401B7564C0C394F7
:10089D00044013756480C39404400B756440C39485
:1008AD0004400375640075BB0A22E564F46002051B
:1008BD0064E573B4070375BB1022743279A687F013
:1008CD00A4C5F0A2F733F8C3E895644002A8648884
:1008DD00228824882588268867227540007541F076
:1008ED0022C2AF75C820A8CCA9CDAA3A30CF010A33
:1008FD0075C824D2AFAB3BAC3C883B893CC3E89B6D
:10090D00F8E99C206908F930670241032160AD3D8B
:10091D008A3DF9EA9DFA600478FF79FFAE3EAF3F5C
:10092D008B3E8C3FC3EC9FFCC3E99CF542A83BA9D1
:10093D003CC3E89EF8E99FF9C3E54113FBE540137D
:10094D00FAE82AF540E93BF54150067540FF75413F
:10095D00FF21AAAA40AB41AC40AD417E047F02C34A
:10096D00EB940440021E1FC3EB940840021E1FC3EC
:10097D00ED13FDEC13FCDEF7C3EA9CFAEB9DFBEFE8
:10098D006009C3E913F9E813F8DFF7EA28FAEB3940
:10099D00FB8A408B4150067BFF8B408B41C3EB9410
:1009AD00025002D2673069047F0321D57892E6FFA9
:1009BD00C3E537948240110FC3E53794A040010F72
:1009CD00C3EF940640027F057E04E541C4540FF940
:1009DD00E541C454F0F8E540C4540F28F8C3E89E2F
:1009ED00FAE99400FB4009C3EA9402EB9400500429
:1009FD007A02E4FB414FAA40AB41EBC4FEEAC4547A
:100A0D000F4EFCC3EA9CFAEB9400FBC3E813C3132F
:100A1D00F8EA28FAEB3400FB8A408B41C3EB9402D1
:100A2D004002C2677804EBC4FE7B00EAC4540F4E4B
:100A3D00FAC3EA98FA4005C3940250027A027892FA
:100A4D00E6FF306002414F855256855357D26043C1
:100A5D00E680C3E49AF8E49BF930670241E9E8FACD
:100A6D00E9FBD3E913FDE813FC88528953C3EF94D6
:100A7D00036038EF20E00DE82CF8E93DF9ECFAEDD4
:100A8D00FB020AA4E828F8E939F9C3E82402F8E9D9
:100A9D003400F97AFE7BFFC3EF9403400E8A548B2A
:100AAD0055884E894F8C508D51611D885489558ABA
:100ABD004E8B4F8C508D51306920C3E533940340DC
:100ACD0019E542A2E713F8E555F4240138400B204F
:100ADD00E7087554FFF42401F555611DE8FAD3E8D4
:100AED0013FC8852C3EF94036020EF20E007E82C3D
:100AFD00F8ECFA6109E8282402F87AFEC3EF9403B2
:100B0D0040088A54884E8C50611D88548A4E8C50F2
:100B1D00E56BC3335002646BF56B30600261277572
:100B2D003402D26043E680E52D54066026A840A924
:100B3D0041C3E913F9E813F8C2AF53E67F7591008D
:100B4D00C3E498F594E499F595759104D26043E664
:100B5D0080D2AF22D265754400752000306B0375CD
:100B6D002040020B80D265754400752040306B0328
:100B7D00752000D2AF7801206722E52D5406600262
:100B8D00C265C3E541940540137802940540087889
:100B9D0003940540027806306902780A206019E551
:100BAD0044601530690AC3E53394034003D5340618
:100BBD00D2AFD26C8151712FD2AF0000C2AF20677E
:100BCD0026E541C3FB940F40027B0FEB24053073E8
:100BDD000123306A02742820620123F930690279F9
:100BED0082E58BC39940B50544E59B5440B5200281
:100BFD00813B30690A08C3E8940A40010861A920C5
:100C0D0065026180C26553E67F759100306710758E
:100C1D0094007595FE759104D26043E6806180AEB7
:100C2D0040AF41C3E49EF594E49FF5958122C3E561
:100C3D00339402500261803065026180D802814F89
:100C4D0061A9C26C53E67F759100855494855595C5
:100C5D00759104854E56854F57D26043E680D2AFCD
:0E0C6D00E52D54066008206A020533020C8B48
:100C7B00306C0D206B0A2065071581158102150E4E
:100C8B002278003064053065027801E53775F0078E
:100C9B00A4F9E5F028F5F0E9A2F013A2F113A2F202
:100CAB0013F537C394785003753778C3E537953808
:100CBB004008D266C290C287C29130600281C5855E
:100CCB005056855157D26043E68022207D11C2AF2A
:100CDB00754302D294C296D2AF759F34020EA5C251
:100CEB00AF754302D294C295D2AF759F34020EA555
:100CFB00307243207D20C2AF754303900142757E55
:100D0B0010C291D295306204D287A119C294D2AF8E
:100D1B00759F35020EA5C2AF754303900142757ED8
:100D2B0010C290D296306204D287A139C294D2AF4E
:100D3B00759F32020EA5207D17C2AF75430390013C
:100D4B001DC291306202D287D2AF759F35020EA5BC
:100D5B00C2AF75430390011DC290306202D287D29D
:100D6B00AF759F32020EA5207D11C2AF754304D221
:100D7B0096C295D2AF759F32020EA5C2AF754304D2
:100D8B00D295C296D2AF759F35020EA53072432015
:100D9B007D20C2AF754305900131757E40C287D26D
:100DAB0094306204D290A1B5C296D2AF759F340233
:100DBB000EA5C2AF754305900153757E20C287D235
:100DCB0094306204D291A1D5C295D2AF759F3402F3
:100DDB000EA5207D17C2AF754305900113C2873056
:100DEB006202D290D2AF759F34020EA5C2AF75438B
:100DFB0005900127C2873062EBD291D2AF759F3439
:100E0B00020EA5207D11C2AF754306D295C294D2B6
:100E1B00AF759F35020EA5C2AF754306D296C2942D
:100E2B00D2AF759F32020EA5307242207D20C2AF29
:100E3B00754301900153757E20C290D296306204A7
:100E4B00D291C151C295D2AF759F32020EA5C2AFDE
:100E5B00754301900131757E40C291D29530620489
:100E6B00D290C171C296D2AF759F35C1A5207D16A8
:100E7B00C2AF754301900127C290306202D291D26A
:100E8B00AF759F32C1A5C2AF754301900113C291DB
:100E9B00306202D290D2AF759F35C266229001119B
:100EAB00757E00C290C287C291D296D294D295C25F
:100EBB006222788076FF0876FF0876FF0876FF08B7
:100ECB00760308760408760B087603087601087615
:100EDB0001788C76010876FF0876FF0876FF087696
:100EEB00FF0876FF0876030876FF0876FF0876FF83
:100EFB000876250876D00876FA0876FA087604087C
:100F0B0076FF08760108760008767A0876FF087671
:100F1B0001087601087600087603227887E6FFC27F
:100F2B0072BF0302D2727888E6C394036008C27D55
:100F3B00E630E102D27DC27E7889E630E102D27ED4
:100F4B00C3EF94026008758E01D273020F5E758E2B
:100F5B0000C273227880E6149000809378A4F67810
:100F6B0081E6149000809378A5F67886E6149000BD
:100F7B008D9378A6F6789CE67538FF75390CB4021C
:100F8B00067538A075390AB40306753882753905AC
:100F9B0078A3E61490009A93F569D1A8222278964B
:100FAB00E6FA7897E6FB7888E6B40305C3EB940E74
:100FBB00FB307F047A007BFFC3EB9AFCC394825017
:100FCB00027C827575000575EC8575F0A4C3E5F0A0
:100FDB00947D40F222D27FF1A912059D7A007B000D
:100FEB007C10120593E55F2AFA74003BFBDCF37C63
:100FFB0004C3EB13FBEA13FADCF7FEC27F120FA953
:10100B0022E5EF20E6037520000520903FFFE52049
:10101B00146006901DFF1460009304600375EF10BD
:10102B007597DE7597AD7581C043FF8012058E7580
:10103B00EF0075A900E5C7240420E70DF521E5B104
:10104B0020E0068521C743B101120EA87580FF75FC
:10105B00A48075F1C275D4BF75907475A57375F2C4
:0F106B007B75D50475A60175E34075E201E4F8C5
:10107A00F6D8FD756B01120EBD121550789886765A
:10108A00753001C2AF1205A71205B712059D1205E8
:10109A00BE12059D1205C512059D1216691205A7F5
:1010AA001205A71205A2C2AF78FA79FA308607D9D3
:1010BA00FBD8F7021C00120F26120F5F120FA8129C
:1010CA000FA978988676120EA875885075891275B8
:1010DA00C82475910475D84075A82275B80275E6BA
:1010EA0090759B80759D0075D1BC75BC5875BB0AFF
:1010FA0075E88075B20112058ED2AF12084753DA2D
:10110A00CF207E0343DA20307E0343DA1043DA012C
:10111A00C2D8C2711205A7D2617B037A0CE55E7050
:10112A00077A0CDB030210B012059D20700302102F
:10113A00B0C270E55FC3940240E1E52F541F856198
:10114A0060F561B560D5DAD5C26153DACF207E0386
:10115A0043DA20307E0343DA10C2D8C27178A2E69D
:10116A007008D274E52F54E0F52FC2757529001264
:10117A0005A2307409C3E529940A4002D275120502
:10118A009378023074027800C3E55F9840F0C2AFEA
:10119A001205B71205B71205B7D2AF1205A7754DDA
:1011AA00007888E6B403024190120593788CE6C36E
:1011BA0094015003021290E530C3940150030212C5
:1011CA0090207435C3E55F94FF5003021290C2AFBA
:1011DA001205CCD2AF1205A2C3E55F940150EFC24B
:1011EA00AF1205B71205981205B7D2AF1205A2C3FE
:1011FA00E55F94FF40E90216EE7F05D27F120FA940
:10120A001205A2C2AFC27F120FA9AE5FC3E55F94F7
:10121A007FD2AF407B12058EC2AF1205CCD2AFDFB0
:10122A00DA120FE0C3EE94057897F61205A71215A5
:10123A00921216717F0AD27F120FA91205A2C2AFAB
:10124A00C27F120FA9AE5FC3E55F947FD2AF50E4AD
:10125A0012058EC2AF1205B71205981205B7D2AFA2
:10126A00DFD4120FE0EE24057896F61205A71215C0
:10127A00921216A01205A2120FA9C3E55F94FF509D
:10128A000221CB0216EEC3E55F954D4003855F4D03
:10129A001205A278017988E7B403027805C3E55FED
:1012AA0098400221ABC2AF1205CC1205CC1205CC74
:1012BA00D2AF1205A7753000E4F531F5320531E5F4
:1012CA0031F470390532789AE67819146012783256
:1012DA0014600D787D14600878FA14600375320082
:1012EA00C3E53298401715327531B478998676C2BB
:1012FA00AF1205CCD2AF789886761205A21205985D
:10130A00E52A700530740201B0780120740278066B
:10131A00C3E55F9840A77888E6C394036003120583
:10132A00A2E52A70030210B0C2AF120EA8E4F52299
:10133A00F523F524F525F526F56AD2AF7885E6C3B7
:10134A0033F568E4F545F546F547F548F549F5738B
:10135A00F52CF52DF53775730875BB1012058E122D
:10136A00084BE5E820ECFBA8BDA9BEE97001F888A6
:10137A007412084F75730875BB107887E6FE7602FB
:10138A00120F267887EEF6C2AF7564FF1208C7857A
:10139A002264852265852266D2AF752201752401F1
:1013AA0075250175260185636C756D017888E6B42B
:1013BA000307C27D307602D27DD268D269753300C6
:1013CA00120E0E120E331208E71208EE1208E71276
:1013DA0008EE1208E70213EFC2AF120F26D2AF755A
:1013EA00730075BB0A120B72120697120C8C120C40
:1013FA00D61208EE120B61306D03120698206703AD
:10140A001207EA306703120831120C8C120CFB1215
:10141A0008EE120B72306D031206D4120C8C120DE8
:10142A00721208EE120B61306D03120732120C8C25
:10143A00120D971208EE120B72306D0312078F12FB
:10144A000C8C120E0E1208EE12084B120B61120CC3
:10145A008C120E3312084F1208EE306932206B2FAD
:0E146A0085676485676585636C756D0179180B
:101478007A0CC3E53399400CC269D26A8A3575641F
:10148800FF021499C3E55F940140030213EF0215AC
:1014980016306A1B206B18E535147004C26A61E2C5
:1014A800F535C3E55F940140030213EF0215167585
:1014B8003600C3E5627882985054307404E52A6097
:1014C8004D7888E6B40317207D0520760781E6303D
:1014D800760281E6206B07D26B856764812E78F0EF
:1014E800306B058567647820C3E54198500261EF49
:1014F800306B1BC26BC27D307602D27DD26A7535E5
:101508001285676461EF0536E55F6002A1197536DB
:1015180000C2AF120EA87887E6FE7602120F267870
:1015280087EEF6E4F522F523F524F525F526F5688A
:10153800C268D2AF12058E120EA8307409C3E53600
:101548009405400201B041C2901A0D78201215D4BA
:10155800E520B45A0CA31215D4E520B4A50302154E
:1015680072120EBD121592021591901A0378807BA3
:101578000A1215D4A308DBF9901A0F788C7B18127D
:1015880015D4A308DBF9901A2722C2AF121613123A
:1015980015ED901A00740E1215D9A374041215D9FA
:1015A800A374141215D9901A0378807B0A1215D8DF
:1015B800A308DBF9901A0F788C7B181215D8A308AA
:1015C800DBF9121626121604901A2722E493F62243
:1015D800E6438F01538FFD75EF0275B7A575B7F117
:1015E800F0538FFE22438F02438F0175EF0275B7C8
:1015F800A575B7F1901A0DF0538FFC22901A0D744F
:101608005AB1D9901A0E74A5B1D9227A3079D07806
:1016180020901A40B1D4E520F709A3DAF7227A30EE
:1016280079D0901A40E7B1D909A3DAF922AB77A8A3
:1016380078BB01027984BB02027985BB03027986F3
:10164800BB04027992BB05027987BB060279A3BB6A
:101658000702799CBB08027988BB09027989E8F7F7
:10166800227C051205A7DCFB22C2AF1205B71205C2
:10167800BE1205C51205CC1205981205B71205BE93
:101688001205C51205CC1205981205B71205BE122F
:1016980005C51205CCD2AF22C2AF1205CC1205C5C2
:1016A8001205BE1205B71205981205CC1205C5120F
:1016B80005BE1205B71205981205CC1205C512050C
:1016C800BE1205B7D2AF22AE77AF78C2AF1205B758
:1016D8001205B71205B7120598DEF21205CC1205ED
:1016E80098DFF8D2AF22D171D169D16975770175C8
:1016F8007801757900D1CF7C05AD5F1205A7C3EDE0
:10170800955F70F5C3E55F9401400AC3E55F94FFF8
:10171800403202172AD135B192D171C2AF75EF109C
:10172800D169DCD50579C3E5799403500280C6D127
:10173800690578E5771490009F93F808C3E57898D1
:10174800500280AED169D1690577C3E577940A5014
:0F17580002809C120EBDB192C2AF75EF10D16925
:0319FD0002100CC9
:101A00000E0414FFFFFFFF03040B0301015AA5019D
:101A1000FFFFFFFFFF03FFFFFF25D0FAFA04FF01DE
:081A2000007AFF01010003FF41
:101A4000234638355F3341232020202020202020CA
:101A500023424C48454C492346383530232020202A
:101A60002020202020202020202020202020202076
:101C0000C2AFC2D37597DE7597AD7581C075A90057
:101C100043FF80752438752503B1C875EF0275E35D
:101C20004043F14053A4BF75D400D2867DFA7803B7
:101C300079E67C10752200752300901DD57B067512
:101C400024987525013086028145208608D8FBD965
:101C5000F9DCF781B7308608D8FBD9F9DCF781B712
:101C6000B188E493A3C39A6004DDC381B7DBDBB121
:101C70007A6002812E7B08E493FAA3B15BDBF87AE9
:101C800030B15B752200752300B17AEAFCEBFDC32D
:101C9000ED94FE400EB17A8A278B28ED30E0048A5D
:101CA000828B83B17A7AC270D8C3ED94FE601350F0
:101CB000CEBD0023EC60097520007521FF020000F5
:101CC0008100A827A9280809D804D90281D4B17EA7
:101CD000EAF281C80D81A3C3ED94035047EDA2E061
:101CE00092007AC5C3E5829400E583941C5092204B
:101CF0000010438F02438F0175B7A575B7F1F0301F
:101D0000001DA827A9280809438F01538FFDD80477
:101D1000D902A11FE275B7A575B7F1F0A3A10E53C3
:101D20008FFC817F7AC1BD030CE493A3FAB13FDC41
:101D3000F8B137817F8181AA22AB23B15BEBFAEA4C
:101D40006222752608C3E52313F523E52213F52245
:101D500050066323A0632201D526EAB1C8B1C87535
:101D6000260AEAF4200102D286300102C286B1C8F6
:101D7000C3134002C201D526EB22B17EEAFB2086C6
:101D800002A17E308602A183752608AE24AF25C34A
:101D9000EF13FFEE13FEB1CCB1C8C3EA13308602D5
:101DA0004480FA30E703632201C3E52313F523E5FA
:101DB0002213F52250066323A0632201D526D9E51C
:101DC0002265236523F52222AE24AF250E0FDEFE09
:101DD000DFFCD20122424C48656C6934373163F82C
:031DE000500601A9
:00000001FF
